:100000000C942A000C9445000C9445000C94450077
:100010000C9445000C949A010C94C7010C94F901BE
:100020000C9445000C9438010C9445000C94450048
:100030000C9445000C946A080C941B030C94450026
:100040000C9445000C9445000C9445000C9445001C
:100050000C94450011241FBECFE5D4E0DEBFCDBF18
:1000600010E0A0E6B0E0E6E3FFE102C005900D92EB
:10007000AC3BB107D9F711E0ACEBB0E001C01D9289
:10008000A735B107E1F70C94AD000C940000CF93B5
:10009000DF93CDB7DEB7E7E3F0E08FE18083E4E301
:1000A000F0E08EEF8083E1E3F0E084E08083E2E340
:1000B000F0E088E38083DF91CF910895CF93DF93C1
:1000C000CDB7DEB721970FB6F894DEBF0FBECDBF18
:1000D000F89480E29EE490934B0180934A01198248
:1000E0002FC08981482F552789819927880F991F0B
:1000F000FC01E252FF4F808191819C0128513C4FCD
:10010000CA01880F991FFC01E65CFE4F31832083F2
:1001100020914A0130914B0189819927880F991FBD
:10012000FC01E65CFE4F80819181A901481B590BBF
:10013000CA0190934B0180934A0189818F5F898323
:100140008981883070F2789421960FB6F894DEBFDA
:100150000FBECDBFDF91CF910895CF93DF93CDB781
:10016000DEB721970FB6F894DEBF0FBECDBF0E9459
:1001700047000E9416010E940D031092390188EB7E
:1001800092E09093D9008093D80086E093E090931A
:10019000DB008093DA0078948091C0008823E1F33B
:1001A0001092C0000E9405060E9444040E94DF06CF
:1001B00000C08091CA00813041F4809139018823C8
:1001C00011F40E945E001092CA008091C300813039
:1001D00021F41092C3000E9439078091C100813040
:1001E00011F41092C1008091C000813011F410927E
:1001F000C0008091BF008130E1F61092BF000E94E4
:100200004C06D7CFCF93DF93CDB7DEB7F894E9E5AF
:10021000F0E089E180837894DF91CF910895CF93C6
:10022000DF93CDB7DEB7DF91CF910895CF93DF9302
:10023000CDB7DEB7E3E5F0E082E08083EFE4F0E005
:100240001082EEE4F0E082E08083EAE4F0E084EF04
:1002500091E091838083E8E4F0E080ED97E0918382
:100260008083E9E5F0E081E08083DF91CF9108951C
:100270001F920F920FB60F9211248F93CF93DF939B
:10028000CDB7DEB78091CF008F5F8093CF00809194
:10029000CF00833029F481E08093C3001092CF0017
:1002A000809138018F5F80933801809138018732C7
:1002B000C9F581E08093C100109238018091CE0091
:1002C0008F5F8093CE008091CE00853029F410920C
:1002D000CE0081E08093C2008091CC008F5F80933C
:1002E000CC008091CC00843641F41092CC0081E0A7
:1002F0008093BE0081E08093C0008091CC00823367
:1003000019F481E08093C0008091CD008F5F8093CD
:10031000CD008091CD008A3029F41092CD0081E08B
:100320008093BF00DF91CF918F910F900FBE0F9000
:100330001F9018951F920F920FB60F9211242F93B2
:100340003F934F935F936F937F938F939F93AF935D
:10035000BF93EF93FF93CF93DF93CDB7DEB7E091D9
:10036000D800F091D9000995DF91CF91FF91EF91DD
:10037000BF91AF919F918F917F916F915F914F91BD
:100380003F912F910F900FBE0F901F9018951F92C5
:100390000F920FB60F9211248F93AF93BF93EF93E9
:1003A000FF93CF93DF93CDB7DEB7A2E3B0E0E2E3F4
:1003B000F0E080818B7F8C93A5E3B0E0E5E3F0E093
:1003C00080818D7F8C9381E08093C9008091BC00F7
:1003D000883019F481E08093CA00DF91CF91FF91BA
:1003E000EF91BF91AF918F910F900FBE0F901F9023
:1003F00018951F920F920FB60F9211242F933F93CF
:100400008F939F93AF93BF93EF93FF93CF93DF931C
:10041000CDB7DEB72297DEBFCDBFA2E3B0E0E2E307
:10042000F0E0808184608C93ECE4F0E01182108233
:10043000A8E4B0E08091BC009927880F991FFC01C7
:10044000E65CFE4F8081918111969C938E93809102
:10045000BC00882339F4A5E3B0E0E5E3F0E0808157
:1004600082608C938091BC00282F33273A832983A4
:1004700089819A8182309105C1F129813A812330A5
:10048000310554F489819A81009789F029813A8154
:1004900021303105D9F04EC089819A818330910590
:1004A00099F129813A8124303105E9F143C0A8E36B
:1004B000B0E0E8E3F0E0808180618C93A8E3B0E0F5
:1004C000E8E3F0E0808181608C9334C0A8E3B0E081
:1004D000E8E3F0E080818E7F8C93A8E3B0E0E8E36E
:1004E000F0E0808182608C9325C0A8E3B0E0E8E36F
:1004F000F0E080818D7F8C93A8E3B0E0E8E3F0E04A
:10050000808184608C9316C0A8E3B0E0E8E3F0E05B
:1005100080818B7F8C93A8E3B0E0E8E3F0E08081FA
:1005200088608C9307C0A8E3B0E0E8E3F0E0808146
:10053000877F8C938091BC008F5F8093BC008091FB
:10054000BC00893010F01092BC002296F894DEBFF7
:10055000CDBFDF91CF91FF91EF91BF91AF919F916F
:100560008F913F912F910F900FBE0F901F90189574
:10057000CF93DF93CDB7DEB78091D0009091D100BB
:100580000097B1F4E6E4F0E0808191819093D70088
:100590008093D600AEE4B0E0EEE4F0E080818F7BA3
:1005A0008C9381E090E09093D1008093D0002BC099
:1005B000E6E4F0E0808191819093D5008093D400AF
:1005C000AEE4B0E0EEE4F0E0808180648C932091B2
:1005D000D4003091D5008091D6009091D700A90128
:1005E000481B590BCA019093D3008093D2001092FC
:1005F000D1001092D0008091D2009091D3009093BE
:100600004D0180934C01DF91CF910895CF93DF93FB
:10061000CDB7DEB7DF91CF910895CF93DF93CDB7FC
:10062000DEB7E7E2F0E01082E6E2F0E08FEE8083F2
:10063000DF91CF9108951F920F920FB60F92112460
:100640002F933F938F939F93EF93FF93CF93DF93DA
:10065000CDB7DEB7E6E2F0E010828091BD009927C9
:10066000E4E2F0E020813181880F991FFC01E25221
:10067000FF4F318320838091BD008F5F8093BD0049
:100680008091BD00873010F01092BD00E7E2F0E0ED
:100690008091BD008083E6E2F0E08FEE8083DF9101
:1006A000CF91FF91EF919F918F913F912F910F905B
:1006B0000FBE0F901F901895CF93DF93CDB7DEB785
:1006C000E9E2F0E080E18083E0E4F0E01082EAE239
:1006D000F0E088E18083E0E4F0E086E88083EBE20C
:1006E000F0E082EC8083DF91CF910895CF93DF9388
:1006F000CDB7DEB721970FB6F894DEBF0FBECDBFE2
:100700008983EBE2F0E080819927807290700097F6
:10071000C1F3ECE2F0E08981808321960FB6F89472
:10072000DEBF0FBECDBFDF91CF910895CF93DF9392
:10073000CDB7DEB726970FB6F894DEBF0FBECDBF9C
:100740009E838D838D819E81DC01FD0101900020BF
:10075000E9F73197CF018A1B9B0B9C838B831A820D
:1007600019820FC029813A818D819E81F901E80F9C
:10077000F91F80810E94760389819A8101969A836C
:10078000898329813A818B819C818217930750F755
:1007900026960FB6F894DEBF0FBECDBFDF91CF9186
:1007A0000895CF93DF93CDB7DEB780916A000E94A2
:1007B000760380916B000E947603DF91CF910895BC
:1007C000CF93DF93CDB7DEB766970FB6F894DEBF51
:1007D0000FBECDBF9E8B8D8B8D899E894AE050E0E8
:1007E0009E012F5F3F4FB9010E941F0FCE0101965E
:1007F0000E94960366960FB6F894DEBF0FBECDBF7B
:10080000DF91CF910895CF93DF93CDB7DEB72297D5
:100810000FB6F894DEBF0FBECDBF8A8387E0898311
:100820001FC08A81482F55278981282F332727FD0C
:10083000309581E090E0022E02C0880F991F0A9443
:10084000E2F7842395231816190624F481E30E9405
:10085000760303C080E30E947603898181508983F7
:1008600089818823F4F680916A000E947603809142
:100870006B000E94760322960FB6F894DEBF0FBE7F
:10088000CDBFDF91CF910895CF93DF93CDB7DEB782
:100890000E947D0463E080E00E94E1058CE690E028
:1008A0000E94830562E081E00E94E10587E790E015
:1008B0000E9483050E947304E0E3F0E080819927A1
:1008C000807290700097C1F70E947D04DF91CF91F4
:1008D0000895CF93DF93CDB7DEB78DE00E94B805C2
:1008E000DF91CF910895CF93DF93CDB7DEB78CE042
:1008F0000E94B805DF91CF910895CF93DF93CDB7D4
:10090000DEB781E00E94B805DF91CF910895CF93C3
:10091000DF93CDB7DEB726970FB6F894DEBF0FBED4
:10092000CDBF9E838D838AE090E09C838B831CC027
:1009300082E390E09A8389830EC08D819E81019726
:100940009E838D838D819E810097B9F789819A81DD
:1009500001979A83898389819A81009799F78B817E
:100960009C8101979C838B838B819C81009701F7ED
:1009700026960FB6F894DEBF0FBECDBFDF91CF91A4
:100980000895CF93DF93CDB7DEB721970FB6F894D4
:10099000DEBF0FBECDBF898389819927817090709A
:1009A000882341F0A5E3B0E0E5E3F0E080818061D9
:1009B0008C9307C0A5E3B0E0E5E3F0E080818F7E93
:1009C0008C938981992782709070009741F0A5E3FC
:1009D000B0E0E5E3F0E0808180628C9307C0A5E39E
:1009E000B0E0E5E3F0E080818F7D8C9389819927E9
:1009F00084709070009741F0A5E3B0E0E5E3F0E08B
:100A0000808180648C9307C0A5E3B0E0E5E3F0E06B
:100A100080818F7B8C938981992788709070009753
:100A200041F0A5E3B0E0E5E3F0E0808180688C93DD
:100A300008C0A5E3B0E0E5E3F0E090818FE789230B
:100A40008C9321960FB6F894DEBF0FBECDBFDF9119
:100A5000CF910895CF93DF93CDB7DEB7A5E3B0E094
:100A6000E5E3F0E0808184608C9381E090E00E9477
:100A70008704A5E3B0E0E5E3F0E080818B7F8C9311
:100A8000DF91CF910895CF93DF93CDB7DEB7229753
:100A90000FB6F894DEBF0FBECDBF8A838A818295E0
:100AA0008F70898389810E94C1040E942A058A81EE
:100AB0000E94C1040E942A0522960FB6F894DEBF58
:100AC0000FBECDBFDF91CF910895CF93DF93CDB708
:100AD000DEB721970FB6F894DEBF0FBECDBF898376
:100AE000A5E3B0E0E5E3F0E0808188608C93898144
:100AF0000E94430521960FB6F894DEBF0FBECDBF0E
:100B0000DF91CF910895CF93DF93CDB7DEB72497D0
:100B10000FB6F894DEBF0FBECDBF9C838B838B8155
:100B20009C81DC01FD0101900020E9F73197CF01A4
:100B30008A1B9B0B8A8319820EC0898199279C018D
:100B40008B819C81F901E80FF91F80810E94650566
:100B500089818F5F898399818A81981770F32496A0
:100B60000FB6F894DEBF0FBECDBFDF91CF910895D1
:100B7000CF93DF93CDB7DEB721970FB6F894DEBFE2
:100B80000FBECDBF898381E090E00E948704A5E37A
:100B9000B0E0E5E3F0E08081877F8C9389810E945B
:100BA0004305A5E3B0E0E5E3F0E0808188608C9345
:100BB00021960FB6F894DEBF0FBECDBFDF91CF9167
:100BC0000895CF93DF93CDB7DEB723970FB6F89490
:100BD000DEBF0FBECDBF8A836B838A81882319F461
:100BE0008B81805889838A81813019F48B8180546C
:100BF000898389810E94B80523960FB6F894DEBFD9
:100C00000FBECDBFDF91CF910895CF93DF93CDB7C6
:100C1000DEB781E090E00E948704A5E3B0E0E5E361
:100C2000F0E08081877F8C9383E00E94C1040E9462
:100C30002A0585E090E00E94870483E00E94C104B9
:100C40000E942A0581E090E00E94870483E00E94D0
:100C5000C1040E942A0582E00E94C1040E942A0564
:100C600081E090E00E94870488E20E94B8058EE04F
:100C70000E94B80581E00E94B80584E890E00E94D7
:100C800083056AE081E00E94E10589E890E00E9426
:100C90008305DF91CF910895CF93DF93CDB7DEB772
:100CA0002C970FB6F894DEBF0FBECDBF8091C40065
:100CB000882309F458C08091C700813009F051C0E1
:100CC0008091C400181634F48091C8008F5F80931F
:100CD000C80005C08091C80081508093C8008091F1
:100CE000C80088231CF483E08093C8008091C8006A
:100CF000843014F01092C8008091C800282F332748
:100D000027FD30953C872B878B859C85813091050D
:100D1000D1F02B853C85223031052CF48B859C85C8
:100D2000009761F01EC02B853C852230310581F093
:100D30008B859C858330910581F013C060E080E055
:100D40000E94E1050EC069E080E00E94E10509C053
:100D500060E081E00E94E10504C069E081E00E945A
:100D6000E1051092C400E0E3F0E0808180728D83A1
:100D70008D81882361F48091C700813041F4809196
:100D8000C800823011F40E94170781E08D838D81A5
:100D9000882351F48091C700843021F40E94A10778
:100DA0000E94DF0681E08D838091C7002C960FB6EC
:100DB000F894DEBF0FBECDBFDF91CF910895CF93E2
:100DC000DF93CDB7DEB781E08093C7001092C800F3
:100DD0000E9469040E947D0460E080E00E94E105B9
:100DE0008EE890E00E94830569E080E00E94E105C2
:100DF00086E990E00E94830560E081E00E94E105C1
:100E00008DE990E00E94830569E081E00E94E105A0
:100E100085EA90E00E9483050E94690460E080E01A
:100E20000E94E1051092C400DF91CF910895CF9305
:100E3000DF93CDB7DEB784E08093C7001092C8007F
:100E40000E947D0469E081E00E94E1058CEA90E067
:100E50000E9483050E94690469E081E00E94E10527
:100E60001092C4000E9473040E948407DF91CF9106
:100E70000895CF93DF93CDB7DEB721970FB6F894DF
:100E8000DEBF0FBECDBF1982F894E0E3F0E08081B1
:100E9000992780719070009711F081E08983E0E3D9
:100EA000F0E08081992788709070009721F0898107
:100EB00093E0892789837894998180916900292F0B
:100EC000281B822F89838981992787FD90958170BE
:100ED0009070882381F080916900982F8981890F13
:100EE000809369008981982F92708091C400890F46
:100EF00081508093C40021960FB6F894DEBF0FBED8
:100F0000CDBFDF91CF910895CF93DF93CDB7DEB7FB
:100F1000F894E0E4F0E01082E9E2F0E081E0808320
:100F2000E0E4F0E08EE88083EAE2F0E088E48083A9
:100F30007894ECE2F0E010821092CB00DF91CF9138
:100F40000895CF93DF93CDB7DEB7F894E0E4F0E0F7
:100F50001082E9E2F0E081E08083E0E4F0E08EE8F6
:100F60008083EAE2F0E010827894DF91CF910895D7
:100F7000CF93DF93CDB7DEB710924E011BC08091A7
:100F80004E01282F332780914E019927880F991FF2
:100F9000FC01E252FF4F808191819695879596954D
:100FA0008795F901EA5FFE4F808380914E018F5F44
:100FB00080934E0180914E01863008F3DF91CF91EE
:100FC0000895CF93DF93CDB7DEB710924E017AC06C
:100FD00080914E019927FC01EA5FFE4F808199279D
:100FE0009093500180934F0120914F013091500117
:100FF00081E591E04AE050E0BC01C9010E941F0F69
:1010000081E591E0DC01FD0101900020E9F73197D5
:10101000CF018A1B9B0B8093560180914E01843037
:1010200030F580914E019927880F991F880F991FDD
:10103000682F80E00E94E10581EB90E00E9483052B
:1010400080914E019927880F991F880F991F982F1B
:1010500080915601292F281B822F8D5F682F80E0F9
:101060000E94E10581E591E00E94830526C0809100
:101070004E019927880F991F880F991F8051682F5B
:1010800081E00E94E10581EB90E00E948305809160
:101090004E019927880F991F880F991F982F8091CB
:1010A0005601292F281B822F8D50682F81E00E9426
:1010B000E10581E591E00E94830580914E018F5FFB
:1010C00080934E0180914E01863008F481CFDF91EC
:1010D000CF9108951F920F920FB60F9211242F9364
:1010E0003F934F935F936F937F938F939F93AF93B0
:1010F000BF93EF93FF93CF93DF93CDB7DEB72C97DA
:10110000DEBFCDBF8091CB00282F332727FD309540
:101110003C872B878B859C8581309105E1F02B8561
:101120003C852230310549F18B859C85009709F07B
:1011300084C0E0E4F0E01082E9E2F0E085E0808342
:10114000ECE2F0E010820E94B8070E94E10781E023
:101150008093CB0072C0E0E4F0E01082E9E2F0E0BE
:1011600081E08083ECE2F0E0108282E08093CB00AB
:101170001092F1001092F00060C080E090E0A0E2D8
:10118000B1E48A839B83AC83BD832BEA3AEA4AE2CB
:1011900050E46A817B818C819D810E94E50ADC019B
:1011A000CB018F839887A987BA8720E030E040E899
:1011B0005FE36F81788589859A850E946F0C88230B
:1011C0000CF003C081E08E8318C020E030E04FE7D0
:1011D00053E46F81788589859A850E94030C1816DF
:1011E0000CF002C01E8209C06F81788589859A85BE
:1011F0000E943409DC01CB018E838E818983898131
:101200008A95F1F78983ACE2B0E02091F00030914B
:10121000F100F901EA5FFE4F80818C93C9010196CC
:101220009093F1008093F0008091F0009091F10094
:101230008233910511F41092CB002C96F894DEBF06
:10124000CDBFDF91CF91FF91EF91BF91AF919F9172
:101250008F917F916F915F914F913F912F910F905F
:101260000FBE0F901F901895EF92FF920F931F9350
:101270007B018C0120E030E040E05FE40E94390C0B
:1012800088237CF020E030E040E05FE4C801B70153
:101290000E94870A0E94A50C6050704080409048D0
:1012A00004C0C801B7010E94A50C1F910F91FF90C7
:1012B000EF900895A0E0B0E0E0E6F9E00C94540F60
:1012C000FC016A019081923008F41BC1DB018C9112
:1012D000823080F0943061F4843009F012C1918141
:1012E000EB018981981709F40CC1E4EBF0E009C126
:1012F000843011F4FB0105C1823091F4923009F081
:1013000000C1EA01DF0188E00D9009928150E1F708
:101310008181FB0191818923E6018983F601F1C076
:10132000923041F362807380EB018A809B80E4807D
:10133000F580068117812C813D814E815F815301AB
:10134000A818B908C501B7FCABC080970CF457C00A
:10135000861497040CF4BEC03401EE24FF248701E8
:101360009181FB018181981709F4A6C0992309F4A2
:101370009CC02E193F09400B510B57FDB0C0E60130
:1013800019827B826A82F6012483358346835783E0
:10139000E6012C813D814E815F8179018A01DA016C
:1013A000C9010197A109B1098F5F9F4FAF4FBF439B
:1013B000F8F4E6016A817B81A8019701220F331FAF
:1013C000441F551F6150704079018A01DA01C9013B
:1013D0000197A109B1098F5F9F4FAF4FBF4360F3E2
:1013E000E6017B836A83F601248335834683578332
:1013F00083E0D6018C9357FD39C0F60182C0861474
:101400009704B4F4C0E0D0E0DA01C90181709070B3
:10141000A070B0705695479537952795282B392B96
:101420004A2B5B2B2196AC16BD0671F78A0C9B1CD0
:10143000681479040CF094CFC0E0D0E05401A618F1
:10144000B708D801C70181709070A070B070169570
:101450000795F794E794E82AF92A0A2B1B2B219683
:10146000AC16BD0671F76A0C7B1C7ACFDA01C90194
:10147000B695A795979587952170307040705070FC
:10148000282B392B4A2B5B2BE6012C833D834E8383
:101490005F838A819B8101969B838A83F60131C099
:1014A000882799278A199B0950CFE21AF30A040B5F
:1014B000150BA801970161CFE60199837B826A82AF
:1014C0002E0D3F1D401F511FF60124833583468397
:1014D00057838ECF20E030E040E050E041CF81E004
:1014E000E60189837B826A825095409530952195EB
:1014F0003F4F4F4F5F4FF601248335834683578319
:1015000047CFCF01EEE0CDB7DEB70C94700FA0E26D
:10151000B0E0EDE8FAE00C945C0F69837A838B838A
:101520009C832D833E834F83588789E1E82EF12CDD
:10153000EC0EFD1EB701CE0101960E94170E8E0122
:101540000F5E1F4FB801CE0105960E94170E8A89C3
:1015500091E089278A8BAE01475F5F4FB801C701D1
:101560000E945A090E94F50CE6E0A0960C94780FB0
:10157000A0E2B0E0EEEBFAE00C945C0F69837A83B2
:101580008B839C832D833E834F83588799E1E92E7B
:10159000F12CEC0EFD1EB701CE0101960E94170E34
:1015A0008E010F5E1F4FB801CE0105960E94170EE7
:1015B000AE01475F5F4FB801C7010E945A090E9400
:1015C000F50CE6E0A0960C94780FA0E2B0E0EBEE0C
:1015D000FAE00C94500F69837A838B839C832D836C
:1015E0003E834F8358878E01075E1F4FB801CE019F
:1015F00001960E94170EF1E1EF2EF12CEC0EFD1E6C
:10160000B701CE0105960E94170E898D823078F0C1
:101610009989923040F420E09A8D8A89981321E0CC
:101620002A8BB701E9C0843051F4923061F020E098
:101630009A8D8A89981321E02A8FB801DDC09430F1
:1016400029F4823041F764EB70E0D6C0823079F340
:10165000923009F32D8D3E8D4F8D58A18D899E8935
:10166000AF89B88D222433242101AA24BB2465012B
:10167000EE24FF24870160E070E00DC06F5F7F4FB4
:101680006032710599F1880F991FAA1FBB1F5695EB
:1016900047953795279520FF19C0280E391E4A1EF9
:1016A0005B1E662477244301281639064A065B062A
:1016B00028F4E1E06E2E712C812C912CAE0CBF1C15
:1016C000C01ED11EA60CB71CC81CD91CEE0CFF1CDA
:1016D000001F111FB7FFD2CFE1E06E2E712C812CBD
:1016E000912CE628F72808291929C8CF8B8D9C8DC5
:1016F0002B893C89820F931F02969C878B871A86C1
:101700009A8D8A89981711F081E08A87D7FE17C0D1
:101710008B859C85A0FE0CC05694479437942794E3
:1017200020E030E040E050E8222A332A442A552ABB
:10173000D694C794B794A79401969C878B8730E082
:10174000A31630E0B30630E0C30630E4D30618F544
:101750008B859C850EC0220C331C441C551C0197A4
:1017600020E0A21620E0B20620E0C20620E4D20665
:1017700080F4AA0CBB1CCC1CDD1C57FEECCF31E066
:10178000632E712C812C912CA628B728C828D92823
:10179000E2CF9C878B87D601C5018F779070A070B0
:1017A000B07080349105A105B10551F0AD86BE86BB
:1017B000CF86D88A83E08987BE01675F7F4F1CC0D0
:1017C000A7FCF4CF211431044104510479F380E4DF
:1017D00090E0A0E0B0E0A80EB91ECA1EDB1E80E8B3
:1017E000682E8FEF782E8FEF882E8FEF982EA62001
:1017F000B720C820D920DACFCB010E94F50CE2E156
:10180000A0960C946C0FA8E1B0E0E9E0FCE00C9429
:101810005C0F69837A838B839C832D833E834F8304
:10182000588781E1E82EF12CEC0EFD1EB701CE01A8
:1018300001960E94170E8E01075F1F4FB801CE015F
:1018400005960E94170E8989823018F42FEF3FEF1A
:101850000BC089858230D0F3B801C7010E94B60E53
:10186000282F332727FD3095C901E6E068960C94B0
:10187000780FA8E1B0E0EFE3FCE00C945C0F698323
:101880007A838B839C832D833E834F83588781E1AA
:10189000E82EF12CEC0EFD1EB701CE0101960E9440
:1018A000170E8E01075F1F4FB801CE0105960E94EB
:1018B000170E8989823018F42FEF3FEF0BC089850E
:1018C0008230D0F3B801C7010E94B60E282F33270B
:1018D00027FD3095C901E6E068960C94780FA8E1E1
:1018E000B0E0E5E7FCE00C945C0F69837A838B83BE
:1018F0009C832D833E834F83588781E1E82EF12C12
:10190000EC0EFD1EB701CE0101960E94170E8E014E
:10191000075F1F4FB801CE0105960E94170E8989F7
:10192000823018F08985823018F421E030E008C058
:10193000B801C7010E94B60E282F332727FD309526
:10194000C901E6E068960C94780FACE0B0E0EBEAF1
:10195000FCE00C94600F69837A838B839C83BE01C7
:101960006B5F7F4FCE0101960E94170E8D818230F2
:1019700061F0823050F0843069F48E81882359F50B
:101980002FEF3FEF4FEF5FE72AC020E030E040E06D
:1019900050E025C02F81388537FDF7CF2F31310535
:1019A00064F78EE190E0821B930B29853A854B8585
:1019B0005C8504C056954795379527958A95D2F74B
:1019C0008E81882361F050954095309521953F4F49
:1019D0004F4F5F4F04C020E030E040E050E8CA01C4
:1019E000B901E2E02C960C947C0F4F925F926F92BB
:1019F0007F928F929F92AF92BF92DF92EF92FF926F
:101A00000F931F9320E030E040E050E0FC01E480C1
:101A1000F58006811781D1808081823038F4D80129
:101A2000C701A061AF77B0706FEFD9C0843009F4FF
:101A30006EC0823009F471C0E114F1040105110592
:101A400009F46BC0828193816FEF823896070CF0A6
:101A50006AC062E87FEF681B790B6A3171050CF090
:101A600080C047015801062E04C0B694A7949794ED
:101A700087940A94D2F744245524320181E090E0FF
:101A8000A0E0B0E004C0880F991FAA1FBB1F6A9591
:101A9000D2F70197A109B109E822F9220A231B23F1
:101AA000E114F1040105110529F061E0462E512CE5
:101AB000612C712C85017401E428F5280629172969
:101AC000D801C7018F779070A070B07080349105F5
:101AD000A105B10509F457C0D801C701CF96A11DD2
:101AE000B11D60E070E08030E0E09E07E0E0AE070E
:101AF000E0E4BE0710F061E070E027E0B695A7953E
:101B0000979587952A95D1F7AF77B07068C080E038
:101B100090E0A0E0B0E06FEF62C080E090E0A0E075
:101B2000B0E060E05CC0803891058CF7BC01615882
:101B30007F4FD801C7018F779070A070B07080344C
:101B40009105A105B105A1F08FE390E0A0E0B0E020
:101B5000E80EF91E0A1F1B1F17FD28C0D801C70178
:101B6000CCCF60E070E080E090E0A0E0B0E0CCCFCF
:101B7000E7FEF2CF80E490E0A0E0B0E0E80EF91ECE
:101B80000A1F1B1FE9CFE7FC18C080E090E060E06F
:101B9000E61660E0F60660E0060760E4160710F05F
:101BA00081E090E0BC01D801C701A7CF1695079549
:101BB000F794E7946F5F7F4FD1CFD801C701805C66
:101BC0009F4FAF4FBF4F60E070E08030E0E09E0776
:101BD000E0E0AE07E0E4BE0708F48FCF8CCF282FFB
:101BE000392F9A2F9F77842F8078892B962F97955E
:101BF000992797958F77482F492B6695852F807861
:101C0000862BD794DD24D7948F77582F5D29CA016E
:101C1000B9011F910F91FF90EF90DF90BF90AF90AF
:101C20009F908F907F906F905F904F900895FC01F0
:101C3000DB01208131819281492F4F7750E0991F3C
:101C40009927991F8381682F660F692B881F882722
:101C5000881FFD018183662309F049C021153105E4
:101C60004105510509F470C082E89FEFFD0193839F
:101C70008283220F331F441F551F220F331F441F1F
:101C8000551F220F331F441F551F220F331F441FA0
:101C9000551F220F331F441F551F220F331F441F90
:101CA000551F220F331F441F551F83E08C93203094
:101CB000F0E03F07F0E04F07F0E45F0790F482E8C0
:101CC0009FEF220F331F441F551F0197203060E004
:101CD000360760E0460760E4560798F3FD019383FA
:101CE0008283FD01248335834683578308956F3FA4
:101CF00071F1862F99278F579040FD01938382833E
:101D000083E08C93220F331F441F551F220F331F74
:101D1000441F551F220F331F441F551F220F331F0F
:101D2000441F551F220F331F441F551F220F331FFF
:101D3000441F551F220F331F441F551F5064248317
:101D4000358346835783089582E08C930895211547
:101D500031054105510519F484E08C93089544FD43
:101D600002C01C92BECF81E08C93BBCFEF92FF925A
:101D70000F931F93CF93DF93FC01DB0180818230AF
:101D800050F09C91923038F0843041F49430B1F0AE
:101D90008181882381F461E070E04BC09430E9F1E7
:101DA0008230A1F09230A1F36181ED018981681741
:101DB00091F0662381F36FEF7FEF3BC0EB018981E8
:101DC000682F77278181681B710933C0923059F5DC
:101DD00060E070E02EC022813381ED018A819B8119
:101DE0008217930734F3281739079CF0E480F580B5
:101DF00006811781FD0124813581468157812E1589
:101E00003F0540075107A8F2E216F306040715073D
:101E1000F8F6662309F0BFCFCECFFB01818188237E
:101E200009F0B9CFC8CFEB018981882309F0B3CF7E
:101E3000C2CFCB01E6E0CDB7DEB70C94780FFB0143
:101E40009F01E8944230C4F04532B4F44A3029F49A
:101E500097FB1EF4909581959F4F642F77270E94E2
:101E6000870F805D8A330CF0895D8193CB010097E9
:101E7000A1F716F45DE251931082C9010C94400F52
:101E8000DC01FC0101900020E9F73297AE17BF0793
:101E900030F47C916081708331976D93F7CF089512
:101EA0002F923F924F925F926F927F928F929F926A
:101EB000AF92BF92CF92DF92EF92FF920F931F9358
:101EC000CF93DF93CDB7DEB7CA1BDB0B0FB6F89409
:101ED000DEBF0FBECDBF09942A88398848885F8449
:101EE0006E847D848C849B84AA84B984C884DF80BA
:101EF000EE80FD800C811B81AA81B981CE0FD11D9E
:101F00000FB6F894DEBF0FBECDBFED010895AA1B3A
:101F1000BB1B51E107C0AA1FBB1FA617B70710F0D4
:101F2000A61BB70B881F991F5A95A9F78095909506
:061F3000BC01CD01089583
:101F36004B2000000000003D00010D0A4550492DD0
:101F46005465737465720056657273696F6E2030DE
:101F56002E3264006875687500416B6B75005050D1
:101F66004D2D4F75740050504D2D496E00444D58FF
:101F76002D4F757400444D582D496E00457869748F
:0C1F86000020200000000000000000000F
:00000001FF
